:020000040000FA
:0400000072303A28F8
:08000800A000030EA100831209
:1000100005191128831601178312B2308100B0012F
:100020002C2883160113831203140B190310A80D37
:10003000A90DAA0DAB0DAC0DAC16FF302C02031DA3
:100040002C28FA302B02031D2C2831152A08AF006A
:100050002908AE002808AD008B100B11210E83007B
:06006000A00E200E0900B5
:0C007400203084008001840A6030040207
:10008000031C3C2851218316FF2390008312831602
:100090000C3085058701831285018701073099009F
:1000A0000030831691009F008312C83083168100B0
:1000B000831231309000003083168C008312103090
:1000C0008B006F2181018E018F010B118B100B10A2
:1000D0008C018B177A20311986203521B30B7828B3
:1000E000031085190314B90DF03039020319DE200D
:1000F00070216A2864003210B00A301F8528AC01D4
:10010000AB01AA01A901A801B00108003111013019
:10011000B7008B132030370783169B001C141A0876
:100120008312A4001030370783169B001C141A0892
:100130008312A300A6000230A606003037078316FC
:100140009B001C141A088312A200A7000130A70606
:100150008B17321CB12822090339A200A309A40974
:10016000A50924082F02031DD82823082E02031DE9
:10017000C62822082D02031DD82801303702031D8E
:10018000C6283D18C6283D143E14692126082E02B3
:10019000031DD82827082D02031DD8280130370257
:1001A000031DD7283D1CD7283D103E146C21D828AC
:1001B000B70A023037020318080089280130B60058
:1001C000B300B400B500B70085018701B1137A20F0
:1001D000B30B0429031085190314B90DF03039024B
:1001E00003192B29B41F8501B41F8701B40B0429FF
:1001F0003708B6080319B60003190229FF30850035
:100200008700B6039630B400311DE7283111321C47
:100210000E292D090339AD00AE09AF092F1CE728BF
:100220008E018F010C1CE7280C102E1EE7288B1363
:1002300020303707BB002F08BA003E2110303707A7
:10024000BB002E08BA003E2100303707BB002D0846
:10025000BA003E218B1785018701B70AB60102302B
:100260003702031CE7286F2108003E1C08003E10DF
:100270001030BB003D08BA003E2108008B133A083D
:1002800083161C159A003B089B0055309D00AA3030
:100290009D009C1464009C184A291C1183128B1722
:1002A0000800831610309B001C141A088312BD002E
:1002B000FF30D4000230D5000C30D600BA30D70061
:1002C0003730D800DA30D9006F30DA00B830DB00D0
:1002D00008000130BD000800850187010800080002
:1002E00001303D05031908005C180516DC18851659
:1002F0005C190514DC1985145C1A8714DC1A0715BF
:100300005C1B0714DC1B87165D180716DD188715A4
:10031000E6300E02031C9629051685160514851471
:100320008714071507148716071687158F080319F2
:1003300008008F01850187015408DE002322D400C4
:100340005508DE002322D5005608DE00541C232267
:10035000D6005708DE00D41C2322D7005808DE0040
:10036000541D2322D8005908DE00D41D2322D900B1
:100370005A08DE00541E2322DA005B08DE00D41E79
:100380002322DB00CA0BCC295408CA00D4185C1401
:10039000D41E5C10D41D5C10CB0BD6295508CB00A5
:1003A000D51ADC14551DDC10551FDC10CC0BE029D0
:1003B0005608CC00561A5C15561F5C11D61D5C11F0
:1003C000CD0BEA295708CD00571ADC15D71FDC11D1
:1003D000D71DDC11CE0BF4295808CE00D81B5C16B3
:1003E000D81F5C12D81C5C12CF0BFE295908CF0015
:1003F000591ADC16591EDC12D91FDC12D00B082A40
:100400005A08D000DA195C17DA1D5C135A1E5C1307
:10041000D10B122A5B08D1005B1ADC175B1EDC13C0
:10042000DB1FDC13D20B1A2A5608D200D51B5D1431
:10043000D71F5D10D30B222A5708D300D61BDD141B
:10044000D81FDD100800C001DE080319DE035E18A6
:100450004014DE1A40144008C0015E1C4014DE1E29
:0A0460004014C005C00C5E0C08003B
:084000000F000300060006009A
:02400E00CC01E3
:10420000010078007A007C007E007B0079007F004E
:104210007D007A0078007E007C00FF00FF00FF0038
:104220000000F200F600FA00FE00F200F600FA00CC
:10423000FE00F200F600FA00FE00FF00FF00FF00A3
:10424000010005000500050005000900090009003E
:1042500009000D000D000D000D00FF00FF00FF0024
:10426000FF00FF00FF00FF00FF00FF00FF00FF0056
:10427000FF00FF00FF00FF00FF00FF00FF00FF0046
:10428000FF00FF00FF00FF00FF00FF00FF00FF0036
:10429000FF00FF00FF00FF00FF00FF00FF00FF0026
:1042A000FF00FF00FF00FF00FF00FF00FF00FF0016
:1042B000FF00FF00FF00FF00FF00FF00FF00FF0006
:1042C000FF00FF00FF00FF00FF00FF00FF00FF00F6
:1042D000FF00FF00FF00FF00FF00FF00FF00FF00E6
:1042E000FF00FF00FF00FF00FF00FF00FF00FF00D6
:1042F000FF00FF00FF00FF00FF00FF00FF00DD00E8
:00000001FF
